:040000008A01032846
:040000008A11D72C5E
:10080000FE00FE1F082C83137E18831700080800C3
:100810000408FE0004308A007E0882070034013498
:1008200000340A34003464340034E83403341034BF
:10083000273425346434003483120313BF000310BB
:10084000003003180130BE003F1C272C282C2C2C14
:100850004008F7007708BE070310C00D0310BF0C57
:10086000BF08031D342C352C242C3E0808008312AD
:100870000313BE000430C0005330BF000130BF027C
:10088000031D432C442C3E2C0130C002031D492C77
:100890004A2C3C2C0130BE02031D4F2C502C3A2C0C
:1008A000080083120313C100410886008A11122533
:1008B0008A110D3083120313C2000130C202031DDE
:1008C000622C632C5D2C08007E088A007F08820061
:1008D00064248A118000840A04087D060319003408
:1008E000FF0A0319FE0A682C0130831203138600E5
:1008F0008A1139258A1164308A1137248A11080037
:1009AE00F001F101F201F301F401F501F601D901B3
:1009BE00DA01DB01DC01DD01DE01DF0183133E30F4
:1009CE00FD000430FE00F430FF00203084008A1158
:1009DE0068248A1183018A11622E9D34FF344134BA
:1009EE0000341734003454340034FF34FF340834E8
:1009FE0000342D34003416340034403400342334A3
:100A0E0000348834FF343034003421340034F5346B
:100A1E00FF344D340034F614760883120313850028
:100A2E001130C0000130C002031D1E2D1F2D192DC7
:100A3E007615760885001130BF000130BF02031D08
:100A4E00292D2A2D242DFB30F7007708F605760880
:100A5E0085001130BE000130BE02031D372D382D2A
:100A6E00322D0800FD30F7007708F6057608831260
:100A7E00031385001130C0000130C002031D482D44
:100A8E00492D432D7615760885001130BF000130B3
:100A9E00BF02031D532D542D4E2DFB30F70077084A
:100AAE00F605760885001130BE000130BE02031D2A
:100ABE00612D622D5C2D080083120313C2000230DB
:100ACE0086008A1139258A1164308A1137248A11D9
:100ADE00283083120313C00042088A111C248A1185
:100AEE00F8008312031343087807C2000310003086
:100AFE0003180130C300962D143086008A11392553
:100B0E008A11213083120313C1000130C102031D6B
:100B1E00912D922D8C2D0130F8007808C3074208D4
:100B2E004302031C9B2D9C2D832D08000B3083123A
:100B3E000313D2005708D401D4075608D301D307A4
:100B4E005B308A1121278A110030F4000030F50045
:100B5E0074085B3E8400831300088A1151248A11A5
:100B6E007408013E5B3E840083138008031DC02D74
:100B7E00C12DC22DD72D0130F4070318F50A003010
:100B8E00F5077508803A83120313D500803055029D
:100B9E00031DD32D04307402031CD62DD72DAF2D7B
:100BAE00080083120313490848040319DF2DE02DB2
:100BBE00102EC5010314C50DEF2D01300310C80D05
:100BCE00C90DFF3E031DE52D0130F8007808C5075D
:100BDE00C91FF22DF32DE42D49084702031DF92DEF
:100BEE0048084602031CFC2DFD2D032E4808C602A4
:100BFE004908031CC703C70201300310C90CC80CF7
:100C0E00FF3E031D042E0130C502031D0F2E102EB4
:100C1E00F32D4708C701C7074608C601C6070800D7
:100C2E00003083120313BE000030BF00440843049B
:100C3E000319222E232E5B2EC0010314C00D322E5B
:100C4E0001300310C30DC40DFF3E031D282E0130CD
:100C5E00F7007708C007C41F352E362E272E013019
:100C6E000310BE0DBF0DFF3E031D372E440842027A
:100C7E00031D432E43084102031C462E472E4E2EC3
:100C8E004308C1024408031CC203C2023E140130D1
:100C9E000310C40CC30CFF3E031D4F2E0130C002C7
:100CAE00031D5A2E5B2E362E3F08C201C2073E0888
:100CBE00C101C1070800031000300318013083166C
:100CCE000313850003100030031801308600031053
:100CDE000030031801308312031385000310003017
:100CEE000318013086008A11BD268A118A117424D8
:100CFE008A110030F0000030F100700883120313E7
:100D0E00D8005807203E840083130008D600840ABA
:100D1E000008D7008A119D258A11FA308A113724CE
:100D2E008A118A1174248A110310003003180130BD
:100D3E0083120313C30000308A1163258A11013018
:100D4E00F0070318F10A0030F1077108803A831298
:100D5E000313D80080305802031DB72E0E307002D8
:100D6E00031CBA2EBB2E842E8A1100283830831213
:100D7E00031386008A1139258A1132308A113724DD
:100D8E008A1138308312031386008A1139258A118D
:100D9E00213083120313C4000130C402031DD82E68
:100DAE00D92ED32E383086008A1139258A1121305A
:100DBE0083120313C5000130C502031DE72EE82E72
:100DCE00E22E383086008A1139258A11213083129D
:100DDE000313C3000130C302031DF62EF72EF12EAE
:100DEE00013086008A1139258A1132308A11372452
:100DFE008A110D308312031386008A1139258A1148
:100E0E00213083120313C1000130C102031D102FC4
:100E1E00112F0B2F063086008A1139258A112130A9
:100E2E0083120313C2000130C202031D1F2F202F95
:100E3E001A2F080083120313D0005330CB00E82F73
:100E4E005108253A03192C2F2D2F392F5108F9004F
:100E5E00500884007908831380000130F900790866
:100E6E00D007E82F0310003003180130CA0000012C
:100E7E000138D2070001FF3852078A1109248A115E
:100E8E00D100003A0319F72F643A0319522F0D3A85
:100E9E000319522FE82F4B08840083130008CD004E
:100EAE00840A0008CE000230F9007908CB07CE1F65
:100EBE00612F622F6B2F0330F9007908CA04CD0918
:100ECE00CE09CD0A0319CE0AD1010314D10D510852
:100EDE00F9007907013EFB008A1109248A11FA00F4
:100EEE00FB0A7B088A1109248A11FB007B084E023B
:100EFE00031D832F7A084D020318862F872F882F04
:100F0E00922F0130F9007908D1075108053A031DD7
:100F1E00912F922F6E2F4A0803390319972F982F6E
:100F2E00A32F2D30F9005008840079088313800018
:100F3E000130F9007908D0075108CC00DE2F4E0899
:100F4E00C201C2074D08C101C1074C08F90079075B
:100F5E00013EFA008A1109248A11C300FA0A7A089E
:100F6E008A1109248A11C4008A1117268A11831343
:100F7E00831203134208C701C7074108C601C607FB
:100F8E000A30C8000030C9008A11D8258A1183138F
:100F9E00831203134608303ED1005108F900500861
:100FAE008400790880000130F9007908D007FF30FD
:100FBE00F9007908CC074C08FF3A031DE72FE82FFC
:100FCE00A62F00010138D2070001FF3852078A11FF
:100FDE0009248A11D100D108031DF62FF72F272FD0
:100FEE000310500884000030031801308313800072
:020FFE000800E9
:00000001FF
